:1000000000308A00A0280000FF00030E8301A10039
:100010007F08A0000A08A8008A01A00E0408A20018
:100020007708A3007808A4007908A5007A08A6003C
:100030007B08A700831383128C308400001C2228C5
:100040000C184F288B1E26280B19392822088400EB
:100050002308F7002408F8002508F9002608FA000C
:100060002708FB0028088A00210E8300FF0E7F0E60
:100070000900FC308100AC0A2C080A3C03184C280B
:100080001F151F19412883161E088312AA001E0877
:10009000AB00FC308100AC010B118A1126280B301B
:1000A0008F00DC308E00AE0A2E08013C0318632856
:1000B0000130AD062D185E2885105F288514831643
:1000C00085108312AE010C108A1126286030831629
:1000D0008F008312B0282B08013C031C7728031DD6
:1000E00075282A088F3C031C77280130A9002B08AB
:1000F000003C03188E28FF3A031D82282A088F3CF3
:1001000003188E282B08033C031C8E28031D8C2803
:100110002A081F3C031C8E280230A9002B08023C31
:1001200003189F28FF3A031D99282A081F3C03182B
:100130009F282B08033C031C9F280430A900D328C8
:1001400084011F308305073083169F008312AC01A2
:100150002D10AE01003083168600831286016628BA
:100160008E3083169F0083121F083839C1389F00D4
:100170000030F8001F08C73978049F008316010873
:10018000C03907388100FC3083128100B5309000FF
:100190000B308F00DC308E00C0308B048B16831642
:1001A0000C1483126B2800308316860083122908F2
:0601B0008600D228630066
:02400E00503F21
:00000001FF
